:020000021000EC
:10F000000C9444F807B004F8030028F9CDFA56F937
:10F0100000000000000000000000000000000000F0
:10F02000000000000C9444F80C9444F80C9444F84C
:10F030000C9444F80C9444F80C9444F80C9444F860
:10F040000C949AFB0C9444F80C9444F80C9444F8F7
:10F050000C9444F80C9444F80C9444F80C9444F840
:10F060000C9444F80C9444F80C9444F80C9444F830
:10F070000C9444F80C9444F80C9444F80C9444F820
:10F080000C9444F80C942CF911241FBECFEFD0E15E
:10F09000DEBFCDBF80E090E00C9463F8000101007A
:10F0A00000000297000100100010000100000200A3
:10F0B000F8941092740017BE1BBE81E085BF15BE88
:10F0C0000C94000008951F93CF93DF93EC0110E0A0
:10F0D0001198199AF89481E085BF82E085BF3DD3ED
:10F0E0008091640080618093640044E150E06CEEA4
:10F0F0007FE087E092E042D390911A029F3F21F097
:10F100008091190288231CF48BE0809319029F3FA1
:10F1100021F0809118028F3F19F485E08093180246
:10F120002091190286E3EBE1F2E0982F11929A9573
:10F13000E9F780931B0231E030931C0230931D02EB
:10F1400010921F0210921E0288EC9AEF90932102F7
:10F150008093200281B38C7F81BB82B38C7F82BB82
:10F1600080E28093700080917400846080937400CA
:10F170008091740080688093740080917400832B68
:10F180008093740080917400806480937400032ED7
:10F1900001C0220F0A94EAF72093720085E091E003
:10F1A000E1E0F1E011920197E9F78FEF9FEFAFEF08
:10F1B000BFEF8093010190930201A0930301B093EC
:10F1C000040110920602E0E0F0E084918F3F11F01C
:10F1D000219711F43093060278942091180230E0C0
:10F1E00044E681B1992796958795982F90959170CF
:10F1F00080910602892B8093060280910602882363
:10F2000011F4222301F150E18091060281114AEFAD
:10F210001F5F141760F010E08091650085278093D0
:10F2200065003F5F3A3018F0312F21112150909145
:10F230000001809100018917E1F380910602882383
:10F2400019F7222309F734DFDF91CF911F91089539
:10F2500081E090E038DF08951F920F920FB60F9271
:10F2600011242F933F934F935F936F937F938F93CB
:10F270009F93AF93BF93EF93FF938BE192E08DD178
:10F2800080917400806880937400FF91EF91BF912A
:10F29000AF919F918F917F916F915F914F913F912E
:10F2A0002F910F900FBE0F901F9018953F924F9285
:10F2B0005F926F927F928F929F92AF92BF92CF9206
:10F2C000DF92EF92FF920F931F93CF93DF93CDB70F
:10F2D000DEB72C970FB6F894DEBF0FBECDBF4C0142
:10F2E0003B01FB018281803BD1F48EE498EFAA2799
:10F2F000BB27880F991FAA1F24E130E0AC01BD0194
:10F30000C301039631D280911902F301838384E112
:10F31000828381E08093060285E190E021C1813BF8
:10F3200079F5DB011496FB01E480FD01F180028197
:10F3300010E09381907C84818D3108F08CE1F301A1
:10F3400082833396992339F499279C01B801A70148
:10F35000CF010AD210C0903831F49927AC01B7011F
:10F36000CF010CD208C0903409F0E1C09927AC015C
:10F37000B701CF0129D2F301828199270196F0C00C
:10F38000823B09F0D7C0DB018C91882309F0E6C0ED
:10F390001496FB01A480FD01B180C280D82E838128
:10F3A000807CFB013380FCEF3F0EECE14E2E4314DA
:10F3B00008F4342C882309F0A7C01496A983BA83D3
:10F3C000E12C7FEFF72E7FEF072F7FEF172FEA203B
:10F3D000FB200C211D21D4012D913D914D915C917B
:10F3E000E216F3060407150719F4332009F076C076
:10F3F000F4018481882309F464C02D833E834F8304
:10F400005887C40105968B839C83412C61E0562E5E
:10F41000612C712C420E531E641E751E49865A863D
:10F420006B867C867FB7F894E199FECF83E0F90183
:10F4300040935B0080936800E8958091680080FDB0
:10F44000FCCF89859A85AB85BC85281739074A0783
:10F450005B0728F561E0AB81BC818D919D91AB8309
:10F46000BC834D805E806F8078840C01F2016092D5
:10F470005B0060936800E8951124D301C2010296F5
:10F48000A11DB11D8D839E83AF83B88749845A84A3
:10F490006B847C8484159505A605B705E0F285E0AC
:10F4A000F90140935B0080936800E89580916800C3
:10F4B00080FDFCCF81E180936800E8957FBFF40177
:10F4C0001482D401ED92FD920D931C93139720E0CA
:10F4D00031E0B801A701C401059646D1332039F1C6
:10F4E000F401808191819501281B390B280D391D6C
:10F4F000832D9927AC0169817A81C901059664D170
:10F5000081E0F401848313C0803841F4832D99276E
:10F51000AC01B501CD01049642D109C0803439F463
:10F52000832D99271496AC01BD01C5014DD180E012
:10F5300090E016C0833B31F4DB018C91882371F499
:10F54000B7DD0CC0843B51F4FB018081882331F48A
:10F55000F89488E181BD88E081BDFFCF8FEF9FEFF8
:10F560002C960FB6F894DEBF0FBECDBFDF91CF91C2
:10F570001F910F91FF90EF90DF90CF90BF90AF90D1
:10F580009F908F907F906F905F904F903F900895E5
:10F59000BC0181E091E08ADE08950F931F93CF9321
:10F5A000DF93EC0180917100887F009174008823C3
:10F5B00009F4A5C0803631F0883621F0803711F08B
:10F5C0008837F1F4803711F0883711F41F8204C0B6
:10F5D000809172008E7F8F8384E090E08B839C8388
:10F5E000629684E2FE0111928A95E9F76297CE0154
:10F5F00044968A879B871C861D866F818C8518C0E0
:10F60000803811F08039B9F4609173008C858232B2
:10F6100030F4EA85FB85E80FF11D608305C0833275
:10F6200018F00F7B1B821C828C858F5F8C878985ED
:10F6300070D0898764C0883809F45CC0883909F4BF
:10F6400059C0803A09F58B819C810497D1F4ED81F2
:10F65000FE81309739F08C858B8BCE0142960995CF
:10F660008B8B01C01B8A2B89222331F0CE0144965B
:10F670008E879F87288B05C01E861F86288B1B823E
:10F680001C821B821C823BC0803B11F0883A89F4AB
:10F690008B819C81892B21F483E090E08B839C8378
:10F6A000198A809172008160682F898532D089879C
:10F6B00002C0883BC9F489899889981710F410E032
:10F6C00010C0891719F419850F7B0BC0EE85FF85D3
:10F6D000E80FF11D8F5F898B1081612F898519D00B
:10F6E0008987109373000BC0803C11F0883C21F493
:10F6F0001B821C82006403C080E090E005C00F778D
:10F700000093740081E090E0DF91CF911F910F9101
:10F710000895682780E027E0962F990F8F5F67FF95
:10F7200003C0692F622701C0692F8830A8F3862F94
:10F73000992708951F920F920FB60F9211248F935D
:10F74000809100018F5F8093000186E082BF8F91DE
:10F750000F900FBE0F901F90189584E083BF12BECC
:10F7600081E087BF789408956BBFFA01DC0102C085
:10F7700007900D9221503040D8F70895411551055A
:10F7800069F0DC01E199FECF7FBB6EBBE09A6F5F51
:10F790007F4F0DB20D9241505040B1F70895411581
:10F7A000510589F0DC018FB7E199FECF7FBB6EBBBD
:10F7B0000D900DBAF894E29AE19A8FBF6F5F7F4F78
:10F7C0004150504089F70895FB01DC0102C00190CF
:0AF7D0000D9241505040D8F7089503
:040000031000F08871
:00000001FF
